:100000000C9434000C943E000C943E000C943E0082
:100010000C943E000C943E000C943E000C943E0068
:100020000C943E000C943E000C943E000C943E0058
:100030000C943E000C943E000C943E000C943E0048
:100040000C943E000C943E000C943E000C943E0038
:100050000C943E000C943E000C943E000C943E0028
:100060000C943E000C943E0011241FBECFEFD8E04C
:10007000DEBFCDBF0E94D3000C9405010C9400009C
:10008000092E000CAA0BBB0B9C01AD0184E0220FD2
:10009000331F441F551F8A95D1F760E074E284EF47
:1000A00090E00E94E300215031093093C500209375
:1000B000C40088E18093C10086E08093C200E0EC38
:1000C000F0E080818D7F808308959091C00095FF3E
:1000D000FCCF8093C60008958091C00087FFFCCFBD
:1000E0008091C6000895EAE7F0E0908197609083E0
:1000F000ACE7B0E09C9190669C939C91907F892B9B
:100100008C93808180688083089580917A008064D8
:1001100080937A0080917A0086FDFCCF80917900EF
:1001200090E0089584B1876084B90895613031F416
:10013000811102C028980895289A0895623031F4F8
:10014000811102C029980895299A0895633029F4ED
:10015000811102C02A9808952A9A08958AB1837F4E
:100160008AB98BB18C608BB90895CF93C82F682F53
:1001700081E00E9496002FEF80E792E021508040BE
:100180009040E1F700C000006C2F80E00E949600D4
:100190002FEF80E792E0215080409040E1F700C0CF
:1001A0000000CF9108950E9492000E94AE0080E866
:1001B00095E20E9440000E946C008136E1F781E0E8
:1001C0000E94B500F8CFA1E21A2EAA1BBB1BFD01AD
:1001D0000DC0AA1FBB1FEE1FFF1FA217B307E40726
:1001E000F50720F0A21BB30BE40BF50B661F771F7E
:1001F000881F991F1A9469F760957095809590955E
:0E0200009B01AC01BD01CF010895F894FFCF22
:00000001FF
